:100000000C9466000C9483000C9483000C94830081
:100010000C9483000C9483000C9483000C94830054
:100020000C9483000C9483000C9483000C94830044
:100030000C9483000C9483000C9483000C94830034
:100040000C9483000C9483000C9483000C94830024
:100050000C9483000C9483000C9483000C94830014
:100060000C9483000C9483000C9483000C94830004
:100070000C9483000C9483000C9483000C948300F4
:100080000C9483000C9483000C9483000C948300E4
:100090000C9483000C9483000C9483000C948300D4
:1000A0000C9483000C9483000C9483000C948300C4
:1000B0000C9483000C9483000C9483000C948300B4
:1000C0000C9483000C9483000C94830011241FBEB5
:1000D000CFEFD8E0DEBFCDBF11E0A0E0B1E0EEEDA4
:1000E000F5E102C005900D92A23BB107D9F721E0DE
:1000F000A2EBB1E001C01D92A43BB207E1F70E9460
:10010000B2030C94ED0A0C940000CF93DF93CDB7AB
:10011000DEB780E890E0FC01108281E890E028E002
:10012000FC01208384E890E0FC0111821082000031
:10013000DF91CF910895CF93DF93CDB7DEB784E8F9
:1001400090E0FC011182108288E890E029E03DE314
:10015000FC013183208386E390E0FC018081882FBD
:1001600090E082709927892B49F086E390E026E39E
:1001700030E0F90120812260FC01208381E890E0D9
:1001800021E830E0F90120812560FC012083000096
:10019000DF91CF910895CF93DF93CDB7DEB786E39C
:1001A00090E0FC018081882F90E082709927892B54
:1001B00049F086E390E026E330E0F90120812260F7
:1001C000FC0120838FE690E028E0FC012083000002
:1001D000DF91CF910895CF93DF93CDB7DEB786E35C
:1001E00090E0FC018081882F90E08270992721E0C7
:1001F000892B09F420E0822FDF91CF910895CF93CE
:10020000DF9300D0CDB7DEB787E690E09A8389838D
:1002100088EC90E0FC01108289EC90E028E1FC0180
:1002200020838AEC90E026E0FC01208389819A817A
:100230008DEC90E0FC0110828CEC90E029813A81F9
:10024000FC01208300000F900F90DF91CF91089563
:10025000CF93DF931F92CDB7DEB789838EEC90E00A
:100260002981FC012083000088EC90E0FC01808162
:10027000882F90E080749927892BB1F388EC90E067
:1002800028EC30E0F90120812064FC01208300008B
:100290000F90DF91CF910895CF93DF93CDB7DEB765
:1002A000000088EC90E0FC0180818823D4F78EEC7C
:1002B00090E0FC018081DF91CF910895CF93DF938F
:1002C00000D000D0CDB7DEB79C838B831A82198211
:1002D0000FC089819A812B813C81820F931FFC0181
:1002E00080810E94280189819A8101969A8389835D
:1002F00089819A812B813C81820F931FFC0180812F
:10030000882339F700000F900F900F900F90DF9126
:10031000CF910895CF93DF93CDB7DEB7A1970FB6F6
:10032000F894DEBF0FBECDBF80E090E0A8ECB2E451
:1003300089839A83AB83BC838CE290E0FC0180814B
:10034000882F90E080749927892B09F07FC00000E6
:100350008CE290E0FC018081882F90E080749927E6
:10036000892BB1F389819A81AB81BC818A879B8774
:10037000AC87BD8720E030E04AE755E46A857B859D
:100380008C859D850E949909DC01CB018E879F8712
:10039000A88BB98B20E030E040E85FE36E857F8575
:1003A000888999890E94F40788232CF481E090E0E1
:1003B0009B8B8A8B3FC020E03FEF4FE757E46E8571
:1003C0007F85888999890E94940918164CF520E048
:1003D00030E040E251E46A857B858C859D850E94F2
:1003E0009909DC01CB01BC01CD010E947208DC013E
:1003F000CB019B8B8A8B0FC080E991E09D8B8C8B0E
:100400008C899D890197F1F79D8B8C8B8A899B89BB
:1004100001979B8B8A8B8A899B89892B69F714C0EA
:100420006E857F85888999890E947208DC01CB01DD
:100430009B8B8A8B8A899B899F8B8E8B8E899F89C8
:100440000197F1F79F8B8E8B84E085C080E290E06E
:10045000FC0180818095837F89878985882309F4C1
:1004600079C0000080E290E0FC0180818F3FD1F7ED
:1004700089819A81AB81BC818D839E83AF83B8874C
:1004800020E030E04AE755E46D817E818F819885D8
:100490000E949909DC01CB01888F998FAA8FBB8FAD
:1004A00020E030E040E85FE3688D798D8A8D9B8D98
:1004B0000E94F40788232CF481E090E09D8F8C8FBC
:1004C0003FC020E03FEF4FE757E4688D798D8A8D7C
:1004D0009B8D0E94940918164CF520E030E040E214
:1004E00051E46D817E818F8198850E949909DC019C
:1004F000CB01BC01CD010E947208DC01CB019D8FB4
:100500008C8F0FC080E991E09F8F8E8F8E8D9F8D95
:100510000197F1F79F8F8E8F8C8D9D8D01979D8F09
:100520008C8F8C8D9D8D892B69F714C0688D798D8A
:100530008A8D9B8D0E947208DC01CB019D8F8C8F70
:100540008C8D9D8D99A388A388A199A10197F1F71E
:1005500099A388A38985A1960FB6F894DEBF0FBE34
:10056000CDBFDF91CF910895CF93DF93CDB7DEB7A5
:1005700063970FB6F894DEBF0FBECDBF898B7B8B20
:100580006A8B1A8219828989882F90E08470992752
:10059000892B11F080E289838989837F8A838BE2AA
:1005A00090E02BE230E0F90130812A812327FC0121
:1005B00020838EE290E02EE230E0F9013081298143
:1005C0002327FC01208320E030E040E85EE364EA7A
:1005D00070ED84EA93E40E9486064A895B8928EEDE
:1005E00033E0429FC001439F900D529F900D112414
:1005F000CC01A0E0B0E0BC01CD010E94A108DC016B
:10060000CB018B839C83AD83BE8320E030E04AE73F
:1006100055E46B817C818D819E810E949909DC016A
:10062000CB018F839887A987BA8720E030E040E824
:100630005FE36F81788589859A850E94F407882316
:100640002CF481E090E09C878B873FC020E03FEF57
:100650004FE757E46F81788589859A850E949409D0
:1006600018164CF520E030E040E251E46B817C81CB
:100670008D819E810E949909DC01CB01BC01CD01D5
:100680000E947208DC01CB019C878B870FC080E938
:1006900091E09E878D878D859E850197F1F79E87D6
:1006A0008D878B859C8501979C878B878B859C8507
:1006B000892B69F714C06F81788589859A850E9496
:1006C0007208DC01CB019C878B878B859C85988B7E
:1006D0008F878F8598890197F1F7988B8F878BE2A9
:1006E00090E02BE230E0F90130812A812327FC01E0
:1006F00020838EE290E02EE230E0F9013081298102
:100700002327FC012083000063960FB6F894DEBF18
:100710000FBECDBFDF91CF910895CF93DF93CDB7BB
:10072000DEB781E290E0FC01108282E290E02FEFE0
:10073000FC0120838AE290E02FEFFC0120838BE212
:1007400090E02FEFFC0120838DE290E020E3FC019C
:1007500020838EE290E02FEFFC0120830000DF91E8
:10076000CF9108958F929F92AF92BF92CF92DF92D6
:10077000EF92FF92CF93DF93CDB7DEB7A5970FB679
:10078000F894DEBF0FBECDBFF8940E9485000E9492
:100790008D030E94FF001A82198284E091E00E947A
:1007A0005E0107C00E944C01882F90E0C0979A8399
:1007B000898389819A810497ACF789819A81181677
:1007C000190684F7A2C189819A8182309105D9F0F6
:1007D0008330910569F1019709F03FC083E090E013
:1007E0009E838D8383E090E09C838B8385E090E003
:1007F00098878F8383E090E09A87898785E090E0EF
:100800009C878B872AC084E090E09E838D8382E062
:1008100090E09C838B8387E090E098878F8383E0D0
:1008200090E09A8789878AE090E09C878B8715C043
:1008300085E090E09E838D8381E090E09C838B83B4
:100840008AE090E098878F8385E090E09A87898797
:100850008FE090E09C878B8700001E861D86188A9B
:100860001F861A8A198A0BC189859A85092E000C60
:10087000AA0BBB0BBC01CD010E94A3086B017C013C
:100880002B853C8589859A85A901481B590BCA018E
:10089000092E000CAA0BBB0BBC01CD010E94A308C2
:1008A0004B015C018D819E810197092E000CAA0BE2
:1008B000BB0BBC01CD010E94A308DC01CB019C0154
:1008C000AD01C501B4010E94F907DC01CB014C0167
:1008D0005D0189899A89092E000CAA0BBB0BBC010A
:1008E000CD010E94A308DC01CB019C01AD01C50133
:1008F000B4010E949909DC01CB01BC01CD010E9429
:10090000DD07DC01CB019C01AD01C701B6010E94EE
:100910007107DC01CB01BC01CD010E946B08DC0139
:10092000CB019B8F8A8F1C8A1B8A37C00E947A0A50
:1009300027E030E0B9010E94060A8D8B8D89833053
:1009400011F487E08D8B8D89282F30E081E090E0D5
:1009500002C0880F991F2A95E2F78C8F8AE00E94C7
:1009600028018D89805D0E9428018AE00E9428016B
:100970009E012F5D3F4F8B899C89820F931F2C8D89
:10098000FC0120838B819C81BC018C8D0E94B40270
:100990008B899C8901969C8B8B8B2B893C898A8DBA
:1009A0009B8D2817390714F28F8198859093B30196
:1009B0008093B2010E949B00198E188E53C01F8A2B
:1009C0001E8A0E94EB008823C1F08091B2019091B1
:1009D000B30101979093B3018093B2010E94CB00C1
:1009E0000E949B002DEC3CEC4CEC5DE364EA70ED66
:1009F00082E893E40E94860606C00E948A01882F3E
:100A000090E09F8B8E8B8E899F89892B39F4809102
:100A1000B2019091B301181619069CF28D859E853E
:100A200001969E878D879E012F5D3F4F888D998D02
:100A3000820F931FFC018081282F30E08E899F89CF
:100A40002817390741F48F8598890196988B8F87ED
:100A50000E94920502C00E94A805888D998D01967A
:100A6000998F888F288D398D8A8D9B8D281739070E
:100A70000CF4A5CF89899A8901969A8B898B29894B
:100A80003A898D819E81281739070CF4EDCE8F8528
:100A90009889092E000CAA0BBB0BBC01CD010E944A
:100AA000A3086B017C018D859E85092E000CAA0B85
:100AB000BB0BBC01CD010E94A308DC01CB019C0152
:100AC000AD01C701B6010E94F907DC01CB018D8F92
:100AD0009E8FAF8FB8A32DEC3CEC4CE45FE36D8DA3
:100AE0007E8D8F8D98A10E949409882354F089816E
:100AF0009A8101969A8389838AE591E00E945E013A
:100B000004C00E946606000005C089819A8103978F
:100B10000CF459CE89819A8103970CF43CCE0E9443
:100B2000460639CECF93DF93CDB7DEB787E691E0A7
:100B30000E945E012DEC3CEC4CEC5DE360E070E06B
:100B40008CED93E40E9486060000DF91CF9108951A
:100B5000CF93DF93CDB7DEB72E970FB6F894DEBFF5
:100B60000FBECDBF82E791E00E945E012DEC3CEC10
:100B70004CE45EE36CE57FEC82E893E40E94860639
:100B800080E090E0A8ECB1E489839A83AB83BC83D6
:100B900020E030E04AE755E469817A818B819C81CD
:100BA0000E949909DC01CB018D839E83AF83B887B6
:100BB00020E030E040E85FE36D817E818F819885A1
:100BC0000E94F40788232CF481E090E09A878987BB
:100BD0003FC020E03FEF4FE757E46D817E818F817A
:100BE00098850E94940918164CF520E030E040E208
:100BF00051E469817A818B819C810E949909DC0191
:100C0000CB01BC01CD010E947208DC01CB019A87A7
:100C100089870FC080E991E09C878B878B859C85B5
:100C20000197F1F79C878B8789859A8501979A8729
:100C3000898789859A85892B69F714C06D817E81A2
:100C40008F8198850E947208DC01CB019A87898781
:100C500089859A859E878D878D859E850197F1F779
:100C60009E878D872DEC3CEC4CE45EE36CE57FECDD
:100C700082E893E40E94860600002E960FB6F89450
:100C8000DEBF0FBECDBFDF91CF910895CF93DF932D
:100C9000CDB7DEB785E891E00E945E0120E030E04C
:100CA00040E05FE360E070E083E893E40E94860642
:100CB00020E030E040E05FE360E070E084EC93E44B
:100CC0000E9486060000DF91CF910895CF93DF93B5
:100CD000CDB7DEB78AE991E00E945E0120E030E006
:100CE00040E05FE360E070E085EA93E40E948606FE
:100CF00020E030E040E05FE360E070E083E993E40F
:100D00000E9486060000DF91CF910895CF93DF9374
:100D1000CDB7DEB76E970FB6F894DEBF0FBECDBF6E
:100D20006F8B788F898F9A8F2B8F3C8F4D8F5E8F33
:100D30002F89388D498D5A8D60E070E080E89FE3FF
:100D40000E94F907DC01CB0120E030E040E050E4F4
:100D5000BC01CD010E94F907DC01CB0120E030E0AD
:100D60004AE754E4BC01CD010E949909DC01CB01A2
:100D70008B839C83AD83BE832F89388D498D5A8D9B
:100D800060E070E080E89FE30E94F907DC01CB019E
:100D90009C01AD016B8D7C8D8D8D9E8D0E94F90720
:100DA000DC01CB01BC01CD010E946B08DC01CB0151
:100DB00098878F831A82198281C08B819C81AD8133
:100DC000BE8189879A87AB87BC8720E030E04AE7FD
:100DD00055E469857A858B859C850E949909DC019B
:100DE000CB018D879E87AF87B88B20E030E040E84D
:100DF0005FE36D857E858F8598890E94F40788233F
:100E00002CF481E090E09A8B898B3FC020E03FEF8B
:100E10004FE757E46D857E858F8598890E949409F8
:100E200018164CF520E030E040E251E469857A85FF
:100E30008B859C850E949909DC01CB01BC01CD0109
:100E40000E947208DC01CB019A8B898B0FC080E96C
:100E500091E09C8B8B8B8B899C890197F1F79C8B04
:100E60008B8B89899A8901979A8B898B89899A8931
:100E7000892B69F714C06D857E858F8598890E94BE
:100E80007208DC01CB019A8B898B89899A899E8BA8
:100E90008D8B8D899E890197F1F79E8B8D8B8EE2CC
:100EA00090E02EE230E0F901308120E12327FC01BF
:100EB000208389819A8101969A8389838F8198857D
:100EC00029813A812817390708F477CF00006E96F8
:100ED0000FB6F894DEBF0FBECDBFDF91CF9108955E
:100EE0005058BB27AA270E9488070C9442090E94E9
:100EF000340938F00E943B0920F039F49F3F19F47F
:100F000026F40C9431090EF4E095E7FB0C940209E9
:100F1000E92F0E94530958F3BA1762077307840731
:100F2000950720F079F4A6F50C948D090EF4E09560
:100F30000B2EBA2FA02D0B01B90190010C01CA0193
:100F4000A0011124FF27591B99F0593F50F4503E3E
:100F500068F11A16F040A22F232F342F4427585F30
:100F6000F3CF469537952795A795F0405395C9F748
:100F70007EF41F16BA0B620B730B840BBAF0915000
:100F8000A1F0FF0FBB1F661F771F881FC2F70EC09F
:100F9000BA0F621F731F841F48F487957795679572
:100FA000B795F7959E3F08F0B0CF9395880F08F05E
:100FB0009927EE0F9795879508950E94750990F0EF
:100FC0009F3748F4911116F40C948E0960E070E09C
:100FD00080E89FE3089526F01B16611D711D811D99
:100FE0000C9408090C9423090E94DE0808F481E09F
:100FF00008950E940D080C9442090E943B0958F084
:101000000E94340940F029F45F3F29F00C94020952
:1010100051110C948E090C9431090E94530968F304
:101020009923B1F3552391F3951B550BBB27AA27A1
:1010300062177307840738F09F5F5F4F220F331FDB
:10104000441FAA1FA9F335D00E2E3AF0E0E832D0A3
:1010500091505040E695001CCAF72BD0FE2F29D0A6
:10106000660F771F881FBB1F261737074807AB0778
:10107000B0E809F0BB0B802DBF01FF2793585F4FED
:101080003AF09E3F510578F00C9402090C948E09B9
:101090005F3FE4F3983ED4F3869577956795B795CF
:1010A000F7959F5FC9F7880F911D9695879597F9DA
:1010B0000895E1E0660F771F881FBB1F6217730753
:1010C0008407BA0720F0621B730B840BBA0BEE1F68
:1010D00088F7E09508950E9472086894B1110C9405
:1010E0008E0908950E945B0988F09F5798F0B92FE8
:1010F0009927B751B0F0E1F0660F771F881F991F4D
:101100001AF0BA95C9F714C0B13091F00E948D0958
:10111000B1E008950C948D09672F782F8827B85F68
:1011200039F0B93FCCF3869577956795B395D9F7A4
:101130003EF490958095709561957F4F8F4F9F4FAE
:101140000895E89409C097FB3EF4909580957095BA
:1011500061957F4F8F4F9F4F9923A9F0F92F96E903
:10116000BB279395F695879577956795B795F11178
:10117000F8CFFAF4BB0F11F460FF1BC06F5F7F4F15
:101180008F4F9F4F16C0882311F096E911C0772327
:1011900021F09EE8872F762F05C0662371F096E830
:1011A000862F70E060E02AF09A95660F771F881FFF
:1011B000DAF7880F9695879597F90895990F0008A3
:1011C000550FAA0BE0E8FEEF16161706E807F90719
:1011D000C0F012161306E407F50798F0621B730BB4
:1011E000840B950B39F40A2661F0232B242B252B35
:1011F00021F408950A2609F4A140A6958FEF811DD8
:10120000811D089597F99F6780E870E060E0089578
:10121000882371F4772321F09850872B762F07C00D
:10122000662311F499270DC09051862B70E060E081
:101230002AF09A95660F771F881FDAF7880F969520
:10124000879597F908959F3F31F0915020F4879545
:1012500077956795B795880F911D9695879597F91E
:1012600008959FEF80EC089500240A94161617063F
:1012700018060906089500240A9412161306140687
:1012800005060895092E0394000C11F4882352F0EA
:10129000BB0F40F4BF2B11F460FF04C06F5F7F4FA2
:1012A0008F4F9F4F089557FD9058440F551F59F089
:1012B0005F3F71F04795880F97FB991F61F09F3F43
:1012C00079F087950895121613061406551FF2CF6C
:1012D0004695F1DF08C0161617061806991FF1CFBC
:1012E000869571056105089408950E945B09A0F038
:1012F000BEE7B91788F4BB279F3860F41616B11DF6
:10130000672F782F8827985FF7CF86957795679511
:10131000B11D93959639C8F30895E894BB276627C5
:101320007727CB0197F908950E94DE0808F48FEF24
:1013300008950E94AC090C9442090E94340938F0C7
:101340000E943B0920F0952311F00C9402090C94A3
:10135000310911240C948E090E94530970F3959F52
:10136000C1F3950F50E0551F629FF001729FBB279C
:10137000F00DB11D639FAA27F00DB11DAA1F649F38
:101380006627B00DA11D661F829F2227B00DA11DEB
:10139000621F739FB00DA11D621F839FA00D611D71
:1013A000221F749F3327A00D611D231F849F600D92
:1013B000211D822F762F6A2F11249F5750409AF0BB
:1013C000F1F088234AF0EE0FFF1FBB1F661F771F47
:1013D000881F91505040A9F79E3F510580F00C9412
:1013E00002090C948E095F3FE4F3983ED4F386958E
:1013F00077956795B795F795E7959F5FC1F7FE2BB2
:10140000880F911D9695879597F9089597FB072E5C
:1014100016F4009407D077FD09D00E941A0A07FC41
:1014200005D03EF4909581959F4F089570956195F4
:101430007F4F0895AA1BBB1B51E107C0AA1FBB1F0A
:10144000A617B70710F0A61BB70B881F991F5A9550
:10145000A9F780959095BC01CD0108958F929F9238
:10146000AF92BF92CF92DF92EF92FF92CF93DF9332
:10147000EC01688179818A819B8161157105810503
:10148000910521F464E279ED8BE597E02DE133EFEE
:1014900041E050E00E948A0A49015A019B01AC01D7
:1014A000A7EAB1E40E94A90A6B017C01ACEEB4EF9B
:1014B000A50194010E94B70ADC01CB018C0D9D1D92
:1014C000AE1DBF1DB7FF03C00197A109B0488883B7
:1014D0009983AA83BB839F77DF91CF91FF90EF9091
:1014E000DF90CF90BF90AF909F908F9008950E9413
:1014F0002E0A089580E091E00E942E0A0895A0E04F
:10150000B0E08093000190930101A0930201B09399
:1015100003010895052E97FB1EF400940E94A10A72
:1015200057FD07D00E94BC0A07FC03D04EF40C9470
:10153000A10A50954095309521953F4F4F4F5F4FF1
:10154000089590958095709561957F4F8F4F9F4F2F
:1015500008950E94DE0AA59F900DB49F900DA49F50
:10156000800D911D11240895B7FF0C94A90A0E94C3
:10157000A90A821B930B0895A1E21A2EAA1BBB1B7A
:10158000FD010DC0AA1FBB1FEE1FFF1FA217B3074F
:10159000E407F50720F0A21BB30BE40BF50B661F65
:1015A000771F881F991F1A9469F760957095809529
:1015B00090959B01AC01BD01CF010895A29FB001A0
:1015C000B39FC001A39F700D811D1124911DB29F77
:0E15D000700D811D1124911D0895F894FFCF18
:1015DE000100000053494D4F4E2047414D450A45ED
:1015EE006E74657220796F7572207374617274698E
:1015FE006E6720646966666963756C7479206C65C4
:10160E0076656C3A0A312E20456173790A322E20A6
:10161E004D6F6465726174650A332E204769766575
:10162E00206D65207061696E2E000A6E65787420DB
:10163E006C6576656C0A000A436F7272656374217D
:10164E000A000A496E636F7272656374206775656E
:10165E0073732E0A000A596F7520626561742074C7
:10166E0068652067616D65210A000A596F75206CE7
:10167E006F6F73652C2074727920616761696E3F9C
:02168E000A0050
:00000001FF
